:100000000C9444050C948C050C948C050C948C0574
:100010000C948C050C948C050C948C050C948C051C
:100020000C948C050C948C050C94DF0E0C94B10F81
:100030000C94851D0C948C050C948C050C948C05EB
:100040000C948C050C948C050C948C050C948C05EC
:100050000C948C050C94F91D0C948C050C948C0557
:100060000C948C050C948C050C948C050C948C05CC
:100070000C948C050C948C050C948C050C948C05BC
:100080000C948C050C948C050C948C050C948C05AC
:100090000C948C050C948C050C948C050C948C059C
:1000A0000C948C050C948C050C948C052D0D540D22
:1000B0004C0E540D4C0EA00DC30D4C0E1A0E290EF5
:1000C000FA12FA12241324137F13B313C115C115A6
:1000D000CA13C115B514B5147B15C1159015AE150D
:1000E000141A082B1518171C12132F0C3080314CC2
:1000F0001E1F20352124222326272D252E802A4924
:10010000807B7A788080802C7E807C807F51504FED
:10011000801D1B7906111905363738107D528080F5
:1001200004160739090D0A0B0F33340E808028801E
:1001300080808080808080808080808080808080BF
:1001400080808080808080808080808080808080AF
:10015000808080808080808080808080808080809F
:100160000A4B6579626F6172642073746172742ED8
:100170000A000A55534220636F6E6669677572659F
:10018000642E0A000A0A544D4B3A613464346631D5
:1001900034392B2F4C5546410A0A002C03460043A4
:1001A000003600360030004300200041006C00742F
:1001B00000200043006F006E00740072006F006C3E
:1001C000006C006500720000000A0354004D004BF3
:1001D000002E0000000403090409028D000501003F
:1001E000A0320904000001030101000921110100EE
:1001F000012240000705810308000A0904010001EB
:1002000003010200092111010001224D00070582AE
:100210000308000A0904020001030000000921117B
:100220000100012236000705830308000A090403C0
:100230000002030000000921110100012222000731
:1002400005840320000107050403200001090404BC
:1002500000010300000009211101000122390007FB
:100260000585032000011201100100000008EDFEC9
:100270000C6600010102000105010906A101050744
:1002800019E029E715002501950875018102050887
:1002900019012905950575019102950175039101D3
:1002A0000507190029F71500250195F87501810248
:1002B000C00631FF0974A1010975150026FF0095DC
:1002C00020750881020976150026FF009520750823
:1002D0009102C005010980A101850216010026379F
:1002E000001A81002AB700751095018100C0050C25
:1002F0000901A1018503160100269C021A01002AAA
:100300009C02751095018100C005010902A1010937
:1003100001A100050919012905150025019505759B
:10032000018102950175038101050109300931152B
:1003300081257F95027508810609381581257F95ED
:100340000175088106050C0A38021581257F950183
:1003500075088106C0C005010906A101050719E05D
:1003600029E7150025019508750181029501750899
:10037000810105081901290595057501910295016D
:10038000750391010507190029FF150026FF009547
:100390000675088100C0636F6E73756D65723A20D3
:1003A000253034580A0073797374656D3A2025300E
:1003B00034580A000A002530325820006B657962F3
:1003C0006F6172643A20004C45443A20253032581F
:1003D0000A00253032583A20253031366225730A1A
:1003E00000722F632030313233343536373839419B
:1003F00042434445460A0064656C5F6B65795F6201
:1004000069743A2063616E27742064656C3A202514
:100410003032580A006164645F6B65795F626974A9
:100420003A2063616E2774206164643A202530327B
:10043000580A004F6E6573686F743A2074696D6571
:100440006F75740A00290A002575002F00257500B4
:100450005D2800256400200025640020002564003C
:1004600020002564007C0025303258006D6F7573C4
:10047000656B6579205B62746E7C782079207620CC
:10048000685D287265702F61636C293A205B006D8E
:100490006B5F776865656C5F74696D655F746F5FCE
:1004A0006D6178203D2025640A006D6B5F7768657B
:1004B000656C5F6D61785F7370656564203D2025B4
:1004C000640A006D6B5F74696D655F746F5F6D6169
:1004D00078203D2025640A006D6B5F6D61785F7345
:1004E00070656564203D2025640A006D6B5F696E50
:1004F00074657276616C203D2025640A006D6B5F27
:1005000064656C6179203D2025640A006D6B5F771E
:100510006865656C5F74696D655F746F5F6D617848
:10052000203D2025640A006D6B5F776865656C5F10
:100530006D61785F7370656564203D2025640A00F5
:100540006D6B5F74696D655F746F5F6D6178203D81
:100550002025640A006D6B5F6D61785F737065655F
:1005600064203D2025640A006D6B5F696E746572BE
:1005700076616C203D2025640A006D6B5F64656CBC
:100580006179203D2025640A000A00257500363A6D
:1005900020776865656C5F74696D655F746F5F6D0A
:1005A00061783A20000A00257500353A20776865A1
:1005B000656C5F6D61785F73706565643A20000AF1
:1005C00000257500343A2074696D655F746F5F6D46
:1005D00061783A20000A00257500333A206D617871
:1005E0005F73706565643A20000A00257500323A31
:1005F00020696E74657276616C286D73293A2000EB
:100600000A00257500313A2064656C6179282A3129
:10061000306D73293A20000A092D2056616C7565EA
:1006200073202D0A004D3E004D25643E20003F0002
:100630007365742064656661756C740A00433E20BE
:100640000077686572652064656C74613A20637533
:1006500072736F723D25642C20776865656C3D254B
:10066000640A53656520687474703A2F2F656E2E86
:1006700077696B6970656469612E6F72672F77693E
:100680006B692F4D6F7573655F6B6579730A000A2F
:10069000092D204D6F7573656B6579202D0A4553C3
:1006A000432F713A09717569740A313A0964656CAE
:1006B0006179282A31306D73290A323A09696E74DA
:1006C000657276616C286D73290A333A096D617819
:1006D0005F73706565640A343A0974696D655F74A7
:1006E0006F5F6D61780A353A09776865656C5F6D93
:1006F00061785F73706565640A363A097768656585
:100700006C5F74696D655F746F5F6D61780A0A7004
:100710003A097072696E742076616C7565730A644B
:100720003A097365742064656661756C74730A7543
:10073000703A092B310A646F776E3A092D310A70CD
:100740006775703A092B31300A7067646F776E3ABB
:10075000092D31300A0A7370656564203D20646597
:100760006C7461202A206D61785F73706565642008
:100770002A2028726570656174202F2074696D6568
:100780005F746F5F6D6178290A003F004D3E200065
:10079000433E20004C25640A000A092D20436F6E59
:1007A000736F6C65202D0A4553432F713A0971759B
:1007B00069740A6D3A096D6F7573656B65790A0026
:1007C0000A092D204D61676963202D0A643A096486
:1007D000656275670A783A096465627567206D61BC
:1007E000747269780A6B3A096465627567206B6593
:1007F00079626F6172640A6D3A0964656275672097
:100800006D6F7573650A763A0976657273696F6EF6
:100810000A733A097374617475730A633A09636FF2
:100820006E736F6C65206D6F64650A302D343A0904
:100830006C61796572302D34284631302D4634296B
:100840000A506175733A09626F6F746C6F61646509
:10085000720A6E3A094E4B524F0A003F004E4B52FD
:100860004F3A206F66660A004E4B524F3A206F6E29
:100870000A0074696D65725F72656164333228299C
:100880003A202530346C580A006B6579626F6172CA
:10089000645F6E6B726F3A2025580A006B6579624F
:1008A0006F6172645F69646C653A2025580A006B59
:1008B0006579626F6172645F70726F746F636F6C81
:1008C0003A2025580A00686F73745F6B6579626F10
:1008D0006172645F6C65647328293A2025580A00A8
:1008E0000A092D20537461747573202D0A00474343
:1008F000433A20352E342E30204156522D4C494259
:10090000433A20322E302E30204156525F4152431E
:10091000483A20617672350A004F5054494F4E5381
:100920003A204C554641204D4F5553454B45592093
:1009300045585452414B455920434F4E534F4C4517
:1009400020434F4D4D414E44204E4B524F204B457E
:10095000594D41505F53454354494F4E203430392F
:10096000360A004255494C443A20613464346631B9
:1009700034392B202831333A33383A3138204D611D
:10098000722031332032303230290A005649443A3D
:100990002030784645454428544D4B2E2920504957
:1009A000443A203078363630432846433636304392
:1009B00020416C7420436F6E74726F6C6C65722989
:1009C000205645523A203078303130300A004445C4
:1009D00053433A20544D4B2E206B6579626F617200
:1009E00064206669726D7761726520666F72204659
:1009F00043363630430A000A092D20566572736962
:100A00006F6E202D0A000A6D6F7573653A206F6650
:100A1000660A000A6D6F7573653A206F6E0A000AE8
:100A20006B6579626F6172643A206F66660A000ACC
:100A30006B6579626F6172643A206F6E0A000A6DAD
:100A400061747269783A206F66660A000A6D617493
:100A50007269783A206F6E0A000A64656275673AB7
:100A6000206F6E0A000A64656275673A206F6666D9
:100A70000A000A0A626F6F746C6F616465722E2ED1
:100A80002E2000433E20000011241FBECFEFDAE0ED
:100A9000DEBFCDBF04B603FE28C08091A4039091B1
:100AA000A503A091A603B091A7038730904BA74060
:100AB000B04BD9F41092A4031092A5031092A60390
:100AC0001092A70314BE0FB6F894A8958091600009
:100AD000886180936000109260000FBE1092010840
:100AE00010920008E0E0F8E3099511E0A0E0B1E021
:100AF000EAEEFCE402C005900D92AE33B107D9F7DF
:100B000023E0AEE3B1E001C01D92A43AB207E1F7E1
:100B10000E94460A0C9473260C940000FF93EF93F6
:100B2000E0913E01F0913F01309709F00995EF9176
:100B3000FF910895FC018591803011F0EFDFFBCF2C
:100B40000895FF27E0E230E247FF0CC0419597FF90
:100B500009C0EDE26095709580959095611D711DBD
:100B6000811D911D27FF02C0219530E350E2AA2785
:100B7000660F771F881F991FAA1FA41710F0A41BC8
:100B800063955A95A9F7AA3008F0A95FA05DAF93C5
:100B9000F395611571058105910541F7ED3211F469
:100BA000EF93F395F21718F43F93F395FBCF8F91E2
:100BB000B5DFFA95E1F70895E991F99185918030D3
:100BC00021F0853219F0AADFF9CF089520E0E894EA
:100BD00055915532C1F3503311F4689455915A33FD
:100BE00048F4505390F3220F022E220F220F200DB3
:100BF000250FF4CF0EF4219589919991533619F36D
:100C0000533729F1533559F1BC0188279927E894C6
:100C10005C3621F48991999168945591543639F450
:100C200046EF7EF077FF0DC08FEF9FEF0AC055377C
:100C30004AE039F0583540E121F0523642E009F0FF
:100C40000895FF93EF937DDFEF91FF91B7CFFF936F
:100C5000EF93FC0181918030B9F360DFFBCFFF930C
:100C6000EF9368DFF1CFDF93CF93CDB7DEB7259653
:100C7000A3DFCF91DF91089561FF02C02D98089501
:100C80002D9A089584B18F6184B93E98469A3F9A0F
:100C90008AB1806F8AB95F9A479884B1806684B9B7
:100CA00085B1806685B9E0E5F1E01192119281E0AD
:100CB000E036F807D1F7E0E4F1E080E591E0119249
:100CC00011928E179F07D9F780E591E09093630109
:100CD0008093620180E491E09093610180936001D0
:100CE00008958F929F92BF92CF92DF92EF92FF92E0
:100CF0000F931F93CF93DF938091600190916101D7
:100D00002091620130916301309361012093600171
:100D10009093630180936201E12CF12CC1E0D0E05B
:100D20000FEF10E085B1982F907EE3FE02C020E126
:100D300001C028E08E2D8770892B822B85B9BE01DA
:100D40000E2C02C0660F771F0A94E2F74B018094C5
:100D5000909440E050E08BB18F7080689A0194E0ED
:100D6000220F331F9A95E1F7822B8BB98AE08A957F
:100D7000F1F700C09A01220F331FE0916001F0915A
:100D80006101E20FF31F8081918186239723892BD4
:100D900009F0479A95E39A95F1F70000B6B45F9889
:100DA000AAE0AA95F1F700C0E0916201F091630119
:100DB0006F01C20ED31ED601369B06C08D919C9149
:100DC00011978821992105C08D919C911197862BAF
:100DD000972B8D939C9386B5CB2CD12C8B1528F01B
:100DE00086B590E08C199D0906C0B6B4C8018C196F
:100DF0009D098B0D911D069768F08091600190917F
:100E00006101820F931FDC018D919C91E20FF31F12
:100E100091838083BAE1BA95F1F700C047985F9A51
:100E20008BE291E00197F1F700C000004F5F5F4F48
:100E30004830510509F08FCFA0916201B091630154
:100E4000E0916001F091610150962D913C91519794
:100E5000808991892817390711F00E94C31D9FEFDF
:100E6000E91AF90AA0E1EA16F10409F05BCF81E082
:100E7000DF91CF911F910F91FF90EF90DF90CF9076
:100E8000BF909F908F90089520916201909163018F
:100E9000E22FF92FE80FF11DE80FF11D80819181FC
:100EA000089581FF02C02E9808952E9A089580918A
:100EB00088020895CF93DF9300D01F92CDB7DEB79D
:100EC0009C0180919B03843019F593E099833B83C7
:100ED0002A839093E9008FEF9091E800815095FD6F
:100EE00006C095ED9A95F1F700008111F5CF80913C
:100EF000E80085FF0DC040E050E063E070E0CE0107
:100F000001960E94FA0B8091E8008E778093E800AA
:100F10000F900F900F90DF91CF910895CF93DF93B3
:100F200000D01F92CDB7DEB720919B03243031F55E
:100F300022E02983805891099B838A8383E08093F0
:100F4000E9008FEF9091E800815095FD06C095ED86
:100F50009A95F1F700008111F5CF8091E80085FFA7
:100F60000DC040E050E063E070E0CE0101960E94C9
:100F7000FA0B8091E8008E778093E8000F900F9035
:100F80000F90DF91CF91089520919B032430F1F4CD
:100F900022E02093E9002FEF3091E800215035FD49
:100FA00006C035ED3A95F1F700002111F5CF2091FB
:100FB000E80025FF0BC040E050E065E070E00E94D3
:100FC000FA0B8091E8008E778093E8000895CF9324
:100FD000DF9320919B03243009F04AC0EC018091FB
:100FE00010018823E1F0809111018823C1F085E090
:100FF0008093E90081E8815049F09091E80095FDE7
:1010000005C09AE29A95F1F700C0F5CF8091E8000B
:1010100085FF2EC040E050E060E270E019C081E042
:101020008093E90081E8815059F09091E80095FDA6
:1010300007C0EFE3F1E03197F1F700C00000F3CF14
:101040008091E80085FF14C040E050E068E070E067
:10105000CE010E94FA0B8091E8008E778093E80021
:1010600080E2FE01A8E6B2E001900D928A95E1F7D8
:10107000DF91CF910895CF93C0916601C1110BC04C
:101080000E94C31D643C79408105910520F081E0F8
:1010900080936601C1E08C2FCF910895FF920F934A
:1010A0001F93CF93DF93D82F0FB607FE83C0809195
:1010B0009B03843081F08091030190E001962091A0
:1010C000050130E0822393232091040130E0821750
:1010D000930709F0CDC00E943B08811110C0809198
:1010E000030190E001962091050130E082239323D3
:1010F0002091040130E08217930709F0B9C00E94E3
:10110000B71D8C01C091E900CF709091EC00892F40
:10111000817090FD80E8C82B84E08093E90085E031
:10112000F82E8091EB0085FD42C08091EB0080FF9E
:101130003EC08091EE0087FF3AC0809104019091FB
:101140000301981709F457C09091E80095FF8EC0ED
:10115000E0910101F0910201E80FF11D20818F5F04
:10116000909105018923809304012093F1008091DF
:10117000E80085FDE2CF8091E80080FFDECF80911E
:10118000E8008E778093E800F0920001D6CF80913E
:10119000030190E001962091050130E08223932322
:1011A0002091040130E08217930709F44CC0CF70FE
:1011B000C093E90040910301842F90E001962091B3
:1011C000050130E0822393232091040130E082174F
:1011D000930709F450C0E0910101F0910201E40F7E
:1011E000F11DD083809103018F5F909105018923C8
:1011F0008093030140C08091E80085FF37C0D09301
:10120000F10021E03091F3008091F20090E0932B07
:10121000892B91F08091E80080FF0EC08091E8005A
:1012200085FF03C01092F100F9CF8091E8008E771E
:101230008093E800F0920001222309F4A8CFCF7038
:10124000C093E90018C080910001882309F4AFCF52
:101250000E94B71D9C018017910711F4890161CF8D
:1012600090910001915090930001F8CF20E0CACFF7
:1012700040910301B0CF80E0DF91CF911F910F919A
:10128000FF90089580919A03811109C00E94640E15
:101290000E94C10E8091E20084608093E200089574
:1012A00010929A0308950895089542E061EC81E058
:1012B0000E94730B42E061EC82E00E94730B42E0FB
:1012C00061EC83E00E94730B42E261EC84E00E94D7
:1012D000730B42E261EC85E00C94730B80919D03EB
:1012E000833009F455C030F4813071F0823009F454
:1012F0008EC008958A3009F47AC08B3009F460C03A
:10130000893009F09CC020C080919C03813A09F08B
:1013100096C08091E800877F8093E8008091A003C9
:101320009091A103892B21F460E288E692E003C04A
:1013300060E080E090E070E00E94450C8091E80061
:101340008B778093E800089580919C03813209F0A7
:1013500076C08091A0039091A103009719F00497A3
:1013600009F06DC08091E800877F8093E80080914C
:10137000E80082FD05C080919B038111F8CF5FC01A
:101380008091F100809388028091E8008B7753C0B0
:1013900080919C03813A09F052C08091A003909102
:1013A000A103892B09F04BC08091E800877F8093CF
:1013B000E8008091E80080FFFCCF8091100136C0EA
:1013C00080919C038132D9F58091A0039091A10373
:1013D000892BA9F58091E800877F8093E8000E941F
:1013E000A80B80919E03809310010C94AA12809107
:1013F0009C03813221F58091E800877F8093E8008B
:101400000E94A80B80919F03809389020895809188
:101410009C03813AA1F48091E800877F8093E800E3
:101420008091E80080FFFCCF809189028093F100D9
:101430008091E8008E778093E8000C94A80B0895C3
:101440008091880280936701109288020E94751132
:101450000C94AA120C94200A0E94431D80919903B7
:10146000882329F00E946C1D81110C945D0B089556
:101470000E94811D809167018093880208950C94D9
:10148000380A08950C94410A0C94410ACF9384B70A
:10149000877F84BF0FB6F894A8958091600088611B
:1014A00080936000109260000FBE90E080E80FB65D
:1014B000F89480936100909361000FBE8EE498E0F1
:1014C0000E94041D86E091E00E94F50F84E891E0FF
:1014D0000E949A050E94440A0E94B4100E94640E61
:1014E0000E94C10E8091E20084608093E2007894B3
:1014F0000E94B61080919B03843019F00E94410A2B
:10150000F9CF82E791E00E949A050E94420A80E6A4
:1015100091E00E949A05C4E080919B03853019F404
:101520000E942C0AF9CF0E94BA102091E400309159
:10153000E50080916401909165012817390761F3F6
:101540008091E4009091E50090936501809364019F
:101550000E943B08882301F380919B038430E1F6CD
:101560008091E9008F702091EC00922F917020FD06
:1015700090E8892BC093E9009091EB0090FF43C065
:101580009091EE0097FF3FC09091040120910301DC
:10159000291709F12091E80025FF1DC0E091010104
:1015A000F0910201E90FF11D30819F5F209105014B
:1015B0009223909304013093F1009091E80095FDFF
:1015C000E3CF9091E80090FFDFCF9091E8009E7705
:1015D0009093E800D9CF9091F3002091F20030E091
:1015E000392B232B81F09091E80090FF0CC0909153
:1015F000E80095FF03C01092F100F9CF9091E80048
:101600009E779093E8008F708093E90085CF292F13
:10161000332723303105C9F060F42130310581F0E2
:101620002230310509F041C08DE890E029ED31E02C
:1016300040C021323105E1F02232310531F135C0AF
:1016400082E190E026E632E034C0992781309105AE
:1016500049F028F0029749F5EBE9F1E005C0E5ED26
:10166000F1E002C0E9ECF1E0849190E09F0121C03B
:1016700065307105D0F4660F771FFB01E75DFE4F03
:101680002081318189E090E014C06530710568F4F3
:10169000FB01EE0FFF1FE15EFE4F20813181FB0158
:1016A000E65EFE4F808190E004C080E090E020E0A4
:1016B00030E0FA0131832083089580E189BD82E121
:1016C00089BD09B400FEFDCF8091D8008F7D809345
:1016D000D8008091E00082608093E0008091E0007B
:1016E00081FDFCCF0895982F973068F59093E9001D
:1016F000981739F07091EC002091ED005091F000B6
:1017000003C0242F762F50E021FD02C09F5FECCF55
:101710003091EB003E7F3093EB003091ED003D7F48
:101720003093ED003091EB0031603093EB0070931B
:10173000EC002093ED005093F0002091EE0027FD87
:10174000E5CF80E008958F708093E90081E00895EF
:1017500080919C0387FF11C08091E80082FD05C045
:1017600080919B038111F8CF11C08091E8008B77A5
:101770000BC080919B03882349F08091E80080FF93
:10178000F8CF8091E8008E778093E800089520914B
:10179000E4003091E50095E64091EC00842F8170E3
:1017A00040FF23C08091E80080FD1DC080919B0315
:1017B000882399F0853099F08091EB0085FD11C068
:1017C0004091E4005091E5002417350729F391502A
:1017D00011F09A01E1CF84E0089582E0089583E05A
:1017E000089581E0089580E008954091E80042FF67
:1017F000DDCF0895CF92DF92EF92FF920F931F9368
:10180000CF93DF93EC018B017A010E94C70B81110A
:1018100033C0E114F10439F0F70180819181081B94
:10182000190BC80FD91FC12CD12C0115110519F1A5
:101830008091E80085FD16C08091E8008E77809346
:10184000E800E114F10449F0F70180819181C80EAC
:10185000D91ED182C08285E00FC00E94C70B8823A9
:1018600021F30AC089918093F10001501109FFEF23
:10187000CF1ADF0ADACF80E0DF91CF911F910F916D
:10188000FF90EF90DF90CF9008952091A2033091C8
:10189000A3032617370748F06115710539F4209125
:1018A000E8002E772093E80001C0B901FC0120E098
:1018B0006115710579F180919B038823F1F18530E1
:1018C000F1F18091E80083FD3CC08091E80082FD49
:1018D0002EC08091E80080FFEBCF2091F300809133
:1018E000F20090E0922B6115710551F0883091055E
:1018F00038F421912093F100615071090196F3CFE2
:1019000021E0089709F020E08091E8008E7780932D
:10191000E800CECF2111CFCF0AC080919B0388234E
:1019200061F0853061F08091E80083FD0AC080910C
:10193000E80082FFF2CF80E0089582E0089583E01E
:10194000089581E008952091A2033091A303261702
:10195000370748F06115710539F42091E8002E77BA
:101960002093E80001C0B901FC0120E06115710578
:1019700091F180919B03882309F440C0853009F4DC
:101980003FC08091E80083FD3DC08091E80082FD6A
:101990002FC08091E80080FFE9CF2091F300809173
:1019A000F20090E0922B6115710559F08830910595
:1019B00040F424912093F100319661507109019611
:1019C000F2CF21E0089709F020E08091E8008E77BF
:1019D0008093E800CBCF2111CCCF0AC080919B032C
:1019E000882361F0853061F08091E80083FD0AC0B2
:1019F0008091E80082FFF2CF80E0089582E00895B0
:101A000083E0089581E008951F93CF93DF93CDB7CE
:101A1000DEB7AA970FB6F894DEBF0FBECDBFECE9D4
:101A2000F3E08091F100819323E0E43AF207C9F7F3
:101A30000E946E098091E80083FF2EC180919C0373
:101A400090919D03492F50E04A30510508F024C180
:101A5000FA01EA5AFF4F0C945926803821F0823857
:101A600009F01AC108C080919803909199039923B5
:101A700089F082600FC08091A0038F70873008F0DA
:101A80000BC18093E9008091EB0085FB882780F9EA
:101A90001092E9009091E800977F9093E80080937E
:101AA000F1001092F100D1C0282F2D7F09F0F4C071
:101AB000882319F0823061F0EFC080919E0381305D
:101AC00009F0EAC0933009F080E0809399032EC0BA
:101AD00080919E0381112AC08091A0038F702FEF07
:101AE000280F263008F0D8C08093E9002091EB0041
:101AF00020FF1CC0933021F48091EB00806214C061
:101B00009091EB0090619093EB0021E030E0A9010F
:101B100002C0440F551F8A95E2F74093EA001092E5
:101B2000EA008091EB0088608093EB001092E9005E
:101B30008091E800877F8093E8000E94A80BACC0EA
:101B40008111AAC010919E031F778091E3008078D5
:101B5000812B8093E3008091E800877F8093E800E9
:101B60000E94A80B8091E80080FFFCCF8091E300E9
:101B700080688093E300111102C082E001C083E01D
:101B800080939B0389C08058823008F085C0809183
:101B90009E0390919F038C3D53E0950779F583E078
:101BA0008A838AE289834FB7F894DE01139620E096
:101BB0003EE051E2E32FF0E050935700E49120FF24
:101BC00003C0E295EF703F5FEF708E2F90E0EA3038
:101BD00010F0C79601C0C0968D939D932F5F24315E
:101BE00049F74FBF8091E800877F8093E8006AE261
:101BF00070E0CE0101960E94450C16C06091A003D2
:101C00007091A103AE014F5F5F4F0E94070BBC01B3
:101C1000892B09F441C09091E800977F9093E800E8
:101C200089819A810E94A30C8091E8008B77809330
:101C3000E80032C0803881F58091E800877F80938A
:101C4000E800809197038093F1008091E8008E77FF
:101C500072CF811121C080919E0390919F0399279B
:101C60000297D4F48091E800877F8093E800809108
:101C70009E03809397030E94A80B80919703811184
:101C800006C08091E30087FD02C081E001C084E0CE
:101C900080939B030E9455098091E80083FF0AC04E
:101CA0008091E800877F8093E8008091EB0080625C
:101CB0008093EB00AA960FB6F894DEBF0FBECDBF9F
:101CC000DF91CF911F9108950E94D20E0E94DA0EEB
:101CD000E0EEF0E0808181608083E8EDF0E08081DB
:101CE0008F77808319BCA7EDB0E08C918E7F8C93A9
:101CF00080818F7E808310929A0308950F931F93A3
:101D0000CF93DF930E94D20E0E94DA0EC8EDD0E08E
:101D100088818F77888388818068888388818F7D98
:101D2000888319BC10929B03109297031092990319
:101D30001092980300EE10E0F80180818B7F808381
:101D400088818160888342E060E080E00E94730BBC
:101D5000E1EEF0E080818E7F8083E2EEF0E0808132
:101D600081608083808188608083F80180818E7F9C
:101D70008083888180618883DF91CF911F910F914B
:101D80000895E8EDF0E080818F7E8083E7EDF0E05C
:101D900080818160808384E082BF81E080939A03A8
:101DA0000C947E0EE8EDF0E080818E7F80831092AF
:101DB000E20008951092DA001092E10008951F9257
:101DC0000F920FB60F9211242F933F934F935F936F
:101DD0006F937F938F939F93AF93BF93EF93FF93F3
:101DE0008091E10082FF0BC08091E20082FF07C07A
:101DF0008091E1008B7F8093E1000E9454098091E3
:101E0000DA0080FF1FC08091D80080FF1BC0809146
:101E1000DA008E7F8093DA008091D90080FF0DC0B8
:101E200080E189BD82E189BD09B400FEFDCF81E07A
:101E300080939B030E94420905C019BC10929B032A
:101E40000E9450098091E10080FF19C08091E2005A
:101E500080FF15C08091E2008E7F8093E200809128
:101E6000E20080618093E2008091D80080628093DC
:101E7000D80019BC85E080939B030E942A0A8091B8
:101E8000E10084FF30C08091E20084FF2CC080E13B
:101E900089BD82E189BD09B400FEFDCF8091D800E3
:101EA0008F7D8093D8008091E1008F7E8093E10048
:101EB0008091E2008F7E8093E2008091E200816059
:101EC0008093E20080919703882311F084E007C09B
:101ED0008091E30087FD02C081E001C083E0809330
:101EE0009B030E943F0A8091E10083FF29C08091FB
:101EF000E20083FF25C08091E100877F8093E100AD
:101F000082E080939B03109297038091E1008E7F83
:101F10008093E1008091E2008E7F8093E2008091C7
:101F2000E20080618093E20042E060E080E00E9495
:101F3000730B8091F00088608093F0000E94530939
:101F4000FF91EF91BF91AF919F918F917F916F9191
:101F50005F914F913F912F910F900FBE0F901F9067
:101F600018951F920F920FB60F9211242F933F9343
:101F70004F935F936F937F938F939F93AF93BF9391
:101F8000CF93DF93EF93FF93C091E900CF708091DF
:101F9000EC00D82FD17080FDD0E81092E90080913C
:101FA000F000877F8093F00078940E94040D1092D7
:101FB000E9008091F00088608093F000CD2BCF7015
:101FC000C093E900FF91EF91DF91CF91BF91AF9165
:101FD0009F918F917F916F915F914F913F912F9141
:101FE0000F900FBE0F901F90189590938F028093C3
:101FF0008E020895E0918E02F0918F02309721F0C9
:102000000190F081E02D099480E00895EF92FF9215
:102010000F931F93CF93DF93E0918E02F0918F0285
:102020003097B1F18C010280F381E02D0995809108
:10203000860382FF2DC080FF04C08CEB93E00E94DA
:102040009A05E80110E286EBE82E83E0F82E8091F5
:10205000860380FF0BC088811F928F93FF92EF92BF
:102060000E9433060F900F900F900F901150219601
:102070001111EDCF8091860380FF0AC084EB93E0BD
:10208000DF91CF911F910F91FF90EF900C949A05E3
:10209000DF91CF911F910F91FF90EF900895E09104
:1020A0008E02F0918F02309721F00480F581E02DAF
:1020B00009940895CF93DF9320918C0230918D0283
:1020C0002817390709F190938D0280938C02E091D3
:1020D0008E02F0918F023097B9F0EC010680F78103
:1020E000E02D09958091860382FF0EC080FF0CC011
:1020F000DF93CF9386EA93E09F938F930E943306FA
:102100000F900F900F900F90DF91CF910895CF9384
:10211000DF9320918A0230918B022817390709F149
:1021200090938B0280938A02E0918E02F0918F024D
:102130003097B9F0EC010084F185E02D099580918C
:10214000860382FF0EC080FF0CC0DF93CF9386E929
:1021500093E09F938F930E9433060F900F900F9000
:102160000F90DF91CF9108950C9476110E94AE1DCF
:102170000C9442068F929F92AF92BF92CF92DF92C1
:10218000EF92FF920F931F93CF93DF9300D000D075
:102190001F92CDB7DEB70E94710601E912E0F12C63
:1021A0008F2D0E9444074C01F801A080B180A82621
:1021B000B926A114B10439F4F3940E5F1F4FF8E06F
:1021C000FF12EECF39C08091860381FD0E94771106
:1021D000E12CCC24C394D12CC5018C219D21892BC9
:1021E00021F1E982FA8221E0C4018C219D21892B11
:1021F00009F420E02B830E94B71D8160782F9D8316
:102200008C8349815A816B818D810E94AD114981F6
:102210005A816B817C818D810E942F1DF801808104
:1022200091818C259D2591838083E394CC0CDD1CCA
:10223000F0E1EF12D1CFC0CF8FEF89838A831B8269
:102240000E94B71D8160782F9D838C8349815A81BC
:102250006B818D810E94AD110E942E1D0E94752000
:102260000E94FA0F90919002891759F10E94FA0F7B
:10227000809390029091860392FF0EC090FF0CC055
:102280001F928F9387EC93E09F938F930E94330666
:102290000F900F900F900F90809190020F900F90E1
:1022A0000F900F900F90DF91CF911F910F91FF90A2
:1022B000EF90DF90CF90BF90AF909F908F900C9455
:1022C0003F1D0F900F900F900F900F90DF91CF91C7
:1022D0001F910F91FF90EF90DF90CF90BF90AF9044
:1022E0009F908F9008950C94510708950895EF9250
:1022F000FF920F931F93CF93DF9381EE93E00E94A1
:102300009A05C0E0D0E083E3E82E81E0F82E02EDEC
:1023100013E08C2F0E9444070E941B1DFF92EF9236
:102320009F938F93DF93CF931F930F930E94330656
:1023300021968DB79EB708960FB6F8949EBF0FBE34
:102340008DBFC830D10529F7DF91CF911F910F9133
:10235000FF90EF90089508950895CF93DF93CDB740
:10236000DEB72B970FB6F894DEBF0FBECDBF942F0C
:102370004F83252F588769877A878B874A855B85A6
:10238000452B31F02F3F31F481E09F3F19F403C01A
:1023900081E001C080E080FD07C04F8158856985DC
:1023A0007A858B850E942F1DDE01119686E0FD0146
:1023B00011928A95E9F785E0FE01379601900D921A
:1023C0008A95E1F749815A816B817C818D819E815B
:1023D0000E94DE182B960FB6F894DEBF0FBECDBF5D
:1023E000DF91CF910895CF93882309F465C0C82F5A
:1023F0008CEF8C0F813A20F080E58C0F8E3248F400
:102400008C2F0E94BF23811157C08C2F0E94C61BA6
:102410000CC080E28C0F883058F4C77081E001C096
:10242000880FCA95EAF70E946B1CCF910C94AF1CE1
:102430008BE58C0F833078F4C53A29F0C63A31F039
:1024400083E890E005C081E890E002C082E890E077
:10245000CF910C945A1088E58C0F853168F5C83AF5
:1024600089F0C93A91F0CA3A99F0CB3AA1F0CC3A46
:10247000A9F0CD3AB1F0CE3AB9F0CF3AC1F080E050
:1024800090E017C082EE90E014C089EE90E011C099
:102490008AEE90E00EC085EB90E00BC086EB90E0FA
:1024A00008C083EB90E005C084EB90E002C087EBAE
:1024B00090E0CF910C948710CF910895882349F133
:1024C0009CEF980F913A20F090E5980F9E3218F407
:1024D0000E94161C0DC090E2980F983058F4877037
:1024E00091E001C0990F8A95EAF7892F0E94711C2B
:1024F0000C94AF1C9BE5980F933020F480E090E0A3
:102500000C945A10885A853120F480E090E00C94A5
:1025100087100895882321F00E946B1C0C94AF1C37
:102520000895882321F00E94711C0C94AF1C08951B
:102530000E948B1C0E945A1C0E94AF1C0E941A21F0
:102540000E94E81F80E090E00E945A1080E090E036
:102550000C9487100E947B1C0C949812CF92DF92EF
:10256000EF92FF920F931F93CF93DF9300D000D091
:102570001F92CDB7DEB76C010E94411D811101C3CE
:1025800085E0F601DE01119601900D928A95E1F742
:10259000F60140815181238134812115310531F0CB
:1025A0005F3F31F481E04F3F19F403C081E001C087
:1025B00080E080FDE6C2F601F280E580E2948FE0E3
:1025C000E82249835A83FB82722F3D832C836F2D2F
:1025D0008D810E94421B8C010E94411B0E94311A76
:1025E000E12FE295EF708E2F90E0FC01E05AFF4F53
:1025F0000C945926812F807F1F70882311F012952B
:10260000107FFF2049F0112309F452C2812F0E944C
:102610007E1C0E94AF1C4CC2802F0E945E121123B0
:1026200009F4AFC2812F0E94841C0F900F900F906D
:102630000F900F90DF91CF911F910F91FF90EF902E
:10264000DF90CF900C94AF1C812F807F1F70803261
:1026500011F01295107F002319F0013009F12BC001
:10266000FF20A9F0EE2059F1F1E0812FEF1228C0F0
:102670000F900F900F900F900F90DF91CF911F91BF
:102680000F91FF90EF90DF90CF900C948E1CEE2076
:1026900021F021E0E21609F474C20E94971C2DC0BB
:1026A000FF20E9F085E08E1508F46BC20E94681CDB
:1026B000812329F022C0FF20F1F0E11015C0812F05
:1026C0000F900F900F900F900F90DF91CF911F916F
:1026D0000F91FF90EF90DF90CF900C948A1294E0CE
:1026E0009E1508F44EC209C0F601858180FFE0C145
:1026F0008F708583E4CFE110EEC1812F61C1812FFE
:1027000086958695837019F08130B9F03AC2FF2022
:1027100019F0C801937002C080E090E00F900F9014
:102720000F900F900F90DF91CF911F910F91FF901D
:10273000EF90DF90CF900C945A10FF2019F0C80151
:10274000937002C080E090E00F900F900F900F9078
:102750000F90DF91CF911F910F91FF90EF90DF903D
:10276000CF900C948710802FFF2019F00E94FB1E41
:1027700002C00E94631F0F900F900F900F900F9058
:10278000DF91CF911F910F91FF90EF90DF90CF904D
:102790000C94E81F812F837009F070C0F110F1C113
:1027A000202F229526952770220F220F602F6F7001
:1027B000862F90E0A0E0B0E06C017D01022E04C005
:1027C000CC0CDD1CEE1CFF1C0A94D2F704FF12C0D7
:1027D0008FE090E0A0E0B0E004C0880F991FAA1F2E
:1027E000BB1F2A95D2F7BC01CD01609570958095ED
:1027F000909503C060E070E0CB01169516951370BC
:102800001230B1F040F56C297D298E299F291130B5
:1028100031F10F900F900F900F900F90DF91CF91AB
:102820001F910F91FF90EF90DF90CF900C94561A6C
:102830006C297D298E299F290F900F900F900F9062
:102840000F90DF91CF911F910F91FF90EF90DF904C
:10285000CF900C94701A0E94561AC701B6010F90BF
:102860000F900F900F900F90DF91CF911F910F91CC
:10287000FF90EF90DF90CF900C943C1AFF2019F05E
:10288000812F817001C08695882309F47AC1202F99
:10289000229526952770220F220F602F6F70862FAA
:1028A00090E0A0E0B0E06C017D01022E04C0CC0CF1
:1028B000DD1CEE1CFF1C0A94D2F704FF12C08FE04F
:1028C00090E0A0E0B0E004C0880F991FAA1FBB1FD2
:1028D0002A95D2F7BC01CD016095709580959095B1
:1028E00003C060E070E0CB011695169513701230AE
:1028F000B1F040F56C297D298E299F29113031F1E5
:102900000F900F900F900F900F90DF91CF911F912C
:102910000F91FF90EF90DF90CF900C941D1B6C29CE
:102920007D298E299F290F900F900F900F900F9067
:10293000DF91CF911F910F91FF90EF90DF90CF909B
:102940000C942F1B0E941D1BC701B6010F900F9006
:102950000F900F900F90DF91CF911F910F91FF90EB
:10296000EF90DF90CF900C940B1B003FC1F128F447
:1029700080E4800F803250F096C0023F09F45EC0C0
:1029800008F449C0033F09F46CC08DC0F02FF0710A
:10299000EF2E812F8F71FF2051F00E94A41A802FFB
:1029A000EE2019F08295807F8BCE8F7089CE0E94A9
:1029B000C51A802FEE2019F08295807F01C08F709C
:1029C0000F900F900F900F900F90DF91CF911F916C
:1029D0000F91FF90EF90DF90CF900C949112FF2019
:1029E000A9F024E02E1508F4CCC0812F8F710F9030
:1029F0000F900F900F900F90DF91CF911F910F913B
:102A0000FF90EF90DF90CF900C94EA1A85E08E153E
:102A100008F4B7C0EACFFF2099F0812F8F710F9093
:102A20000F900F900F900F90DF91CF911F910F910A
:102A3000FF90EF90DF90CF900C94A41AFF2069F3E1
:102A4000812F8F710F900F900F900F900F90DF914B
:102A5000CF911F910F91FF90EF90DF90CF900C944A
:102A6000C51AFF2089F0812F8F710F900F900F9062
:102A70000F900F90DF91CF911F910F91FF90EF90EA
:102A8000DF90CF900C948F1A0F900F900F900F90B3
:102A90000F90DF91CF911F910F91FF90EF90DF90FA
:102AA000CF900C948A1AFF2099F0EE2009F4B5CF4C
:102AB000802F0F900F900F900F900F90DF91CF917C
:102AC0001F910F91FF90EF90DF90CF900C94F31136
:102AD000EE2009F4B5CF802F0F900F900F900F903C
:102AE0000F90DF91CF911F910F91FF90EF90DF90AA
:102AF000CF900C945E12412F4F70602FC6010E9440
:102B0000751E0F900F900F900F900F90DF91CF9147
:102B10001F910F91FF90EF90DF90CF900C948C1944
:102B200001112FC0FF2069F10E94AA129FEFE0E778
:102B3000F2E09150E040F040E1F700C000000F905B
:102B40000F900F900F900F90DF91CF911F910F91E9
:102B5000FF90EF90DF90CF900C941E1E412F4F708E
:102B6000602FC6010F900F900F900F900F90DF9184
:102B7000CF911F910F91FF90EF90DF90CF900C9429
:102B8000781E0F900F900F900F900F90DF91CF91C4
:102B90001F910F91FF90EF90DF90CF9008951F93BA
:102BA000CF93DF9300D000D01F92CDB7DEB7942F24
:102BB0004983252F5A836B837C838D834C815D8170
:102BC000452B31F02F3F31F481E09F3F19F403C0D2
:102BD00081E001C080E0182F117080FD31C0498173
:102BE0005A816B817C818D810E94421B292F229505
:102BF0002F702C3030F42A30A0F42250223030F0E4
:102C000022C02C30C9F02F30B9F01DC0853A28F40D
:102C10008430C0F4823028F415C090E2980F9830C8
:102C200088F0883E30F4803E68F48450813A58F44D
:102C300009C0803F41F406C093FB112710F903C07F
:102C400010E001C011E0812F0F900F900F900F90B6
:102C50000F90DF91CF911F910895CF93DF9300D014
:102C600000D01F92CDB7DEB70F900F900F900F904E
:102C70000F90DF91CF910895CF93DF9300D000D0D4
:102C800000D0CDB7DEB726960FB6F894DEBF0FBEE4
:102C9000CDBFDF91CF9108951F93CF93DF93C09164
:102CA000A10216E08091A202C81799F0D0E01C9F03
:102CB000F0011D9FF00D1124ED55FD4F4081518114
:102CC00062817381848195810E943C162196C77030
:102CD000E9CFDF91CF911F9108954091D302509198
:102CE000D4026091D5027091D6028091D702909162
:102CF000D8020C943C16CF938091D80282958F70A5
:102D000009F05FC08091D502882309F45AC08091F0
:102D1000A102B091A2027091D302A091D40240917D
:102D2000D6025091D70291E07F3F09F090E0692FE1
:102D3000C6E08B1709F445C04115510521F0AF3F9E
:102D400021F020E003C021E001C0262F90E020FD0B
:102D500035C0C89FF001C99FF00D1124ED55FD4FFE
:102D600021812A132BC02081271328C02281211101
:102D700025C0238134812417350710F421503109EF
:102D8000241B350B2C323140C8F42091D8022F700F
:102D900020612093D80226E0289FF001299FF00DA2
:102DA0001124E855FD4F80818F708061808383ED11
:102DB00092E00E94AE12CF910C944C16019687704F
:102DC000B8CFCF910895AF92BF92CF92DF92EF929A
:102DD000FF920F931F93CF93DF93CDB7DEB7619729
:102DE0000FB6F894DEBF0FBECDBF7C0185E0F701C2
:102DF000DE011D9601900D928A95E1F7D7014C9165
:102E000011965C9111971296DC90129713960D9182
:102E10001C9114973091D3026091D4028091D60214
:102E20009091D702009731F06F3F31F421E03F3F9E
:102E300019F403C021E001C020E0B22FB170BB2E15
:102E400020FD76C1A090D502AA2009F4D1C020911E
:102E5000D8020817190750F0F801E81BF90BCF0149
:102E6000CC24C3948C329140D0F009C080959095C9
:102E7000800F911FCC24C3948C32914080F0C12CE0
:102E8000207F09F0A1C0702F198B088B6D2D8989C7
:102E90000E942D1683ED92E00E94AE12BDC0822FDB
:102EA000807F09F056C0561315C0431313C0CD2CB4
:102EB000D11010C02F7020612093D8020E946D168F
:102EC00083ED92E00E94AE128091D802D701159650
:102ED0008C9362C10115110531F05F3F31F481E03F
:102EE0004F3F19F403C081E001C080E080FD03C0C2
:102EF00081E08D2502C080E090E0B82FB170CB2E2C
:102F000080FF1CC08091A1022091A20236E08217AE
:102F100009F41FC190E0389FF001399FF00D112492
:102F2000ED55FD4F6181561306C06081461303C005
:102F30006281D61203C001968770E9CFCD2CDD20C7
:102F400009F42AC18091D80281608093D802C12CF3
:102F500023C1561308C0431306C0D11004C080918A
:102F6000D802D701B9C04D875E87DF86702F198BD5
:102F7000088B6D2D89890E94CF15882399F1DD205A
:102F800089F12091D802822F82958F7090E002976C
:102F900074F08091D3029091D40298878F83198620
:102FA0001B870A872C87CE0107960E94AE1286E007
:102FB000F701A3EDB2E001900D928A95E1F70E942E
:102FC0007B160E946D1611C0561781F14D875E87E2
:102FD000DF86702F198B088B6D2D89890E94CF1584
:102FE000811138C0C7010E94AE12CC24C394D4C052
:102FF0000817190708F446C0F801E81BF90BCF01C0
:103000008C32914008F446C0C12C702F198B088B6C
:103010006D2D89890E942D16E3EDF2E086E0DF0137
:103020001D928A95E9F70E946D16B6C04313CECF64
:10303000D110CCCF8091D802F7018583C7010E94BF
:10304000AE1286E0E3EDF2E0DF011D928A95E9F72A
:10305000CA2CA2C0DD2031F22091D802822F8295A5
:103060008F7090E002970CF4A2CF8091D3029091E0
:10307000D4029A8389831B821D830C832E83CE0105
:10308000019693CF80959095800F911F8C3291403F
:1030900008F0BACFCD2CDD2009F4A4CF561333C0ED
:1030A000431331C02091D80220FD24C0822F829585
:1030B0008F70482F50E041155105E1F0D70115966A
:1030C0002C9315974F30510549F08F5F982F9295AB
:1030D000907F822F8F70892B15968C93C7010E9449
:1030E000AE1286E0F701A3EDB2E001900D928A9551
:1030F000E1F799CF86E0F701A3EDB2E001900D92E0
:103100008A95E1F749C04D875E87DF86702F198B5E
:10311000088B6D2D89890E94CF15811148CF809130
:10312000D80281608093D802C7010E94AE1234C0D9
:10313000DD2009F457CF4D875E87DF86702F198B0E
:10314000088B6D2D89890E94CF15882309F44ACFF9
:103150002ECF702F198B088B6D2D89890E94421BF1
:10316000292F22952F70223028F49F7039F0811179
:1031700005C00BC0243028F49F7049F4805E88306D
:1031800020F0C7010E94AE12BC2CCB2C05C0F70169
:103190009581907F99F7F9CF8C2D61960FB6F894B1
:1031A000DEBF0FBECDBFDF91CF911F910F91FF907A
:1031B000EF90DF90CF90BF90AF9008951F93CF9383
:1031C000DF93CDB7DEB72C970FB6F894DEBF0FBEF6
:1031D000CDBF4F83588769877A878B879C87CE01BD
:1031E00007960E94E3168823D1F09F8188852A855F
:1031F0003B85232B31F08F3F31F481E09F3F19F461
:1032000003C081E001C080E080FD47C04F81588548
:1032100069857A858B859C850E943C163EC086E038
:10322000FE013796DE01119601900D928A95E1F725
:10323000FF81E8856A857B856115710531F0EF3F77
:1032400031F481E0FF3F19F403C081E001C080E068
:1032500080FD23C02091A20230E0C9010196877051
:1032600099274091A10250E084179507F1F1F98365
:10327000EA837D836C8396E0929FD001939FB00D8B
:103280001124AD55BD4FFE01319601900D929A95D6
:10329000E1F78093A2020E944C1616E08091A102F1
:1032A0009091A202891771F1189FC00111248D55C8
:1032B0009D4F0E94E316882329F1E091A1021E9FF1
:1032C000F0011124ED55FD4F4081518162817381E0
:1032D000848195810E943C168091A10290E0019624
:1032E000877099278093A102D9CF0E94AA121092C9
:1032F000A2021092A102E3EDF2E086E0DF011D924E
:103300008A95E9F72C960FB6F894DEBF0FBECDBFB5
:10331000DF91CF911F910895DF92EF92FF920F936B
:103320001F93CF93DF93FC01892B09F488C0E12C14
:10333000F12CDD24D394EF0121968491853709F493
:1033400060C058F4843708F04EC0843008F068C07C
:103350008130D1F0823071F172C0883709F45BC0DE
:1033600050F4863709F453C0873709F068C08E2DB2
:103370000E94781C52C09CE7980F903708F05FC0FD
:103380008F770E945E124EC08F010E5F1F4FFE01AD
:10339000849190E2980F983050F48770FD2D01C011
:1033A000FF0F8A95EAF78F2F0E947E1C15C00E949E
:1033B000F31114C08F010E5F1F4FFE01849190E244
:1033C000980F983068F48770FD2D01C0FF0F8A9523
:1033D000EAF78F2F0E94841C0E94AF1CE80122C0D4
:1033E0000E945E12FBCFCF010296FE01C491CC2356
:1033F00061F0EFE9FFE03197F1F700C00000C15044
:10340000F6CFCF010296FE01F490EC010BC00E94B2
:10341000681CE82E07C00E947B1C0E94AF1C02C0E3
:103420000E94F3118F2D882341F0EFE9FFE03197DF
:10343000F1F700C000008150F6CFFE017CCFDF9194
:10344000CF911F910F91FF90EF90DF9008956093BF
:10345000590370935A0380935B0390935C030C941D
:103460003C06089560935D0370935E0380935F0351
:10347000909360030C943E1D0F931F9300915D0386
:1034800010915E0320915F0330916003602B712BDC
:10349000822B932B60935D0370935E0380935F0395
:1034A000909360031F910F910C943E1D0F931F93F7
:1034B00000915D0310915E0320915F0330916003E2
:1034C000602371238223932360935D0370935E03D3
:1034D00080935F03909360031F910F910C943E1DA6
:1034E0000F931F9300915D0310915E0320915F0382
:1034F00030916003602771278227932760935D03D3
:1035000070935E0380935F03909360031F910F910C
:103510000C943E1D60E070E0CB010C94271A0F93D1
:103520001F9341E050E060E070E08A019B0104C01D
:10353000000F111F221F331F8A95D2F7C901B8014E
:103540001F910F910C94271A0F931F9341E050E0A5
:1035500060E070E004C0440F551F661F771F8A9516
:10356000D2F78091590390915A03A0915B03B091D7
:103570005C038A019B01082B192B2A2B3B2BC901C9
:10358000B8011F910F910C94271A0F931F9341E0DC
:1035900050E060E070E004C0440F551F661F771FC5
:1035A0008A95D2F740955095609570958091590312
:1035B00090915A03A0915B03B0915C038A019B0137
:1035C000082319232A233B23C901B8011F910F9116
:1035D0000C94271A0F931F9341E050E060E070E0D5
:1035E00004C0440F551F661F771F8A95D2F780913C
:1035F000590390915A03A0915B03B0915C038A0137
:103600009B01082719272A273B27C901B8011F91C9
:103610000F910C94271A0F931F9300915903109147
:103620005A0320915B0330915C03602B712B822B3A
:10363000932B1F910F910C94271A0F931F930091B6
:10364000590310915A0320915B0330915C0360236E
:103650007123822393231F910F910C94271A0F93A8
:103660001F930091590310915A0320915B033091ED
:103670005C0360277127822793271F910F910C9479
:10368000271A08958F929F92AF92BF92DF92EF9286
:10369000FF920F931F93CF93DF9300D000D01F9220
:1036A000CDB7DEB76B837C838D838A018C819D814E
:1036B000892B31F01F3F31F481E04F3F19F403C0F3
:1036C00081E001C080E080FF03C080E090E04DC059
:1036D0008B818823D1F18090590390905A03A09058
:1036E0005B03B0905C0380915D0390915E03A091B9
:1036F0005F03B0916003882A992AAA2ABB2A8FE126
:10370000E82EF12CD501C4010E2C04C0B695A79566
:10371000979587950A94D2F780FD06C081E0E81A54
:10372000F10880F7D12C07C0DE2CB8018E2D0E9445
:103730004D1E019799F380E1189FF0011124E75283
:10374000FD4FE00FF11DD08209C080E1189FF0010C
:103750001124E752FD4FE00FF11DD08009831A8339
:1037600069817A818D2D0E944D1E0F900F900F90D0
:103770000F900F90DF91CF911F910F91FF90EF90DD
:10378000DF90BF90AF909F908F900895909110011F
:10379000992379F190911101992359F1982F9695D8
:1037A000969596959F31A1F0E0911201F091130149
:1037B000E90FF11D877021E030E0A90102C0440F3C
:1037C000551F8A95E2F7CA019181892B818308955B
:1037D0009091860390FF29C01F928F9385E194E01A
:1037E0009F938F930E9433060F900F900F900F902E
:1037F00008952091120130911301F90132969FEF43
:1038000040E05191851789F09F3F19F4511101C093
:10381000942F4F5F4E31A9F79F3F39F0F901E90F1F
:10382000F11D97FDFA9582830895089590911001F6
:10383000992381F190911101992361F1982F969527
:10384000969596959F31A9F0E0911201F0911301A0
:10385000E90FF11D877021E030E0A90102C0440F9B
:10386000551F8A95E2F7CA0180959181892381834A
:1038700008959091860390FF1CC01F928F9387EF4D
:1038800093E09F938F930E9433060F900F900F90B9
:103890000F900895E0911201F09113019F01225EB3
:1038A0003F4F9281891301C012823196E217F307CC
:1038B000C1F7089581E090E0E0911201F0911301C9
:1038C000E80FF91F1082019680329105A9F708953B
:1038D00080918503089590918503892B80938503BA
:1038E0000895809590918503892380938503089599
:1038F0008093850308951092850308959091840321
:10390000892B809384030895809590918403892363
:103910008093840308951092840308958093630331
:103920000E94B71D909362038093610308951092E3
:103930006303109262031092610308958091120153
:1039400090911301FC0131969C01205E3F4F80E075
:10395000919191118F5FE217F307D1F70895E091EC
:103960001201F0911301809185038083E09112018F
:10397000F0911301908180918403892B8083809141
:1039800063038823D9F10E94B71D20916103309110
:1039900062038217930748F00E94B71D20916103CC
:1039A00030916203821B930B0AC00E94B71D2091C5
:1039B00061033091620320953095820F931F8C3202
:1039C000914070F08091860380FF08C083E394E00B
:1039D0009F938F930E9433060F900F900E94971C25
:1039E000E0911201F0911301908180916303892B82
:1039F00080830E949E1C81110E94971C809112015D
:103A0000909113010C94061090933F0180933E0116
:103A100008958295982F937344E0949F9001112408
:103A20008C7C86958695282B822F8575880F2A7A1F
:103A30002695822B0895CF93DF93D92F0E94091DDD
:103A4000C82F8D2F0E94091D2C2F30E0322F2227E6
:103A5000A901482BCA01DF91CF9108950895CF9312
:103A6000DF9300D000D01F92CDB7DEB70F900F903C
:103A70000F900F900F90DF91CF91089508950C94BF
:103A8000731180E0089580919B03843021F110929E
:103A9000870320E488E190E00FB6F894A89580931E
:103AA00060000FBE2093600083B7817F846083BF76
:103AB00083B7816083BF7894889583B78E7F83BFF7
:103AC0000FB6F894A895809160008861809360009B
:103AD000109260000FBE0895CF930E94AB110E9418
:103AE00071060E94AC11C0E08C2F0E944407892B04
:103AF00029F4CF5FC830C1F780E001C081E0CF91E9
:103B000008950E9475110C94AA121F920F920FB67D
:103B10000F9211248F939F93AF93BF93809187034C
:103B2000811113C08091880390918903A0918A0329
:103B3000B0918B034196A11DB11D80938803909392
:103B40008903A0938A03B0938B03BF91AF919F9198
:103B50008F910F900FBE0F901F90189582E084BD3B
:103B600093E095BD9AEF97BD80936E0008952FB7AF
:103B7000F8948091880390918903A0918A03B09171
:103B80008B032FBF08952FB7F8946091880370912D
:103B9000890380918A0390918B032FBF0895CF9260
:103BA000DF92EF92FF920F931F932FB7F8944091FB
:103BB00088035091890360918A0370918B032FBF12
:103BC0006A017B01EE24FF248C0120E030E0C01666
:103BD000D106E206F30610F4415051099A01281B60
:103BE000390BC9011F910F91FF90EF90DF90CF909B
:103BF00008951F920F920FB60F9211248F939F93E7
:103C0000AF93BF938091880390918903A0918A0319
:103C1000B0918B030196A11DB11D809388039093F1
:103C20008903A0938A03B0938B03BF91AF919F91B7
:103C30008F910F900FBE0F901F9018950E94640EE9
:103C4000F89487E797E7909301088093000887E04E
:103C500090EBDC018093A4039093A503A093A603AB
:103C6000B093A7039CE088E10FB6F894A8958093E1
:103C700060000FBE90936000FFCFE82FF0E080E17E
:103C8000989FE00DF11D1124E052FF4F8491982F71
:103C900092959F708F7097700895CF93C82FCB0126
:103CA0000E943D1E40E1949F90011124282B203852
:103CB00031051CF080E090E016C09770E92FF0E02D
:103CC00098E0C99FE00DF11D112494E0EE0FFF1F55
:103CD0009A95E1F78F70E80FF11DEE0FFF1FE0508E
:103CE000F84985919491CF91089580E090E00895EE
:103CF000089580918E0380FF0BC06091170185E0CD
:103D0000689FB001112475956795759567952BC0CF
:103D100081FF09C06091170185E0689FB0011124FF
:103D20007595679520C082FF07C06091170185E0F7
:103D3000689FB001112417C090918F039923D1F08F
:103D400060911601961788F72091170185E0289F4A
:103D500090011124929FA001939F500D112470E0B7
:103D6000CA010E9445266038710540F4611571054D
:103D700019F406C065E070E0862F08958FE7089576
:103D800081E0089580918E0380FF08C06091150145
:103D900070E0759567957595679521C081FF06C0A0
:103DA0006091150170E07595679519C082FF04C098
:103DB0006091150170E010C090918F03992399F0E4
:103DC000609114019617A0F780911501899FC00199
:103DD000112470E00E9445266038710540F4611599
:103DE000710519F406C061E070E0862F08958FE731
:103DF000089581E00895803F21F40E94791E819505
:103E000004C0813F29F40E94791E80939203089593
:103E1000823F21F40E94791E819504C0833F29F4DA
:103E20000E94791E809391030895893F19F40E949E
:103E3000C21E05C08A3F31F40E94C21E8195809344
:103E4000930308958B3F21F40E94C21E819504C004
:103E50008C3F29F40E94C21E809394030895843FEE
:103E600021F480919003816017C0853F21F48091F7
:103E70009003826011C0863F21F48091900384609A
:103E80000BC0873F21F480919003886005C0883F74
:103E900031F48091900380618093900308958D3F69
:103EA00021F480918E0381600BC08E3F21F48091BC
:103EB0008E03826005C08F3F29F480918E03846059
:103EC00080938E030895803F39F48091920387FF99
:103ED0006CC01092920369C0813F29F480919203D3
:103EE0001816BCF362C090919103823F29F497FFAA
:103EF0005CC01092910359C0833F19F41916CCF39A
:103F000054C0893F41F48091930318160CF04DC0C2
:103F1000109293034AC08A3F29F48091930387FF4C
:103F200044C0F6CF8B3F39F48091940387FF3DC0A6
:103F3000109294033AC08C3F29F480919403181690
:103F4000BCF333C0843F21F4809190038E7F17C06F
:103F5000853F21F4809190038D7F11C0863F21F42D
:103F6000809190038B7F0BC0873F21F48091900359
:103F7000877F05C0883F31F4809190038F7E8093C6
:103F8000900313C08D3F21F480918E038E7F0BC070
:103F90008E3F21F480918E038D7F05C08F3F29F4E1
:103FA00080918E038B7F80938E038091910381118A
:103FB0000EC08091920381110AC0809193038111F8
:103FC00006C080919403811102C010928F0308955E
:103FD0008091860383FF7EC08CE694E00E949A0560
:103FE000809190031F928F9387E694E09F938F9325
:103FF0000E94330685E694E00E949A058091910321
:10400000282F082E000C330B3F938F9382E694E009
:104010009F938F930E94330680E694E00E949A0556
:1040200080919203282F082E000C330B3F938F931F
:104030008DE594E09F938F930E9433068BE594E087
:104040000E949A0580919303282F082E000C330BB1
:104050003F938F9388E594E09F938F930E9433065C
:1040600086E594E00E949A0580919403282F082EFB
:10407000000C330B3F938F9383E594E09F938F93D2
:104080000E94330680E594E00E949A0580918F0398
:104090001F928F938DE494E09F938F930E94330639
:1040A0008BE494E00E949A0580918E031F928F9377
:1040B00088E494E09F938F930E94330685E494E014
:1040C0000E949A058DB79EB74C960FB6F8949EBF86
:1040D0000FBE8DBF80E993E00E944F100E94B71D74
:1040E00090938D0380938C0308951F93CF93DF9358
:1040F00080918C0390918D030E94CF1DAC01909113
:104100008F03992321F02091180130E006C02091FF
:1041100019018AE0289F900111244217530708F4DF
:1041200085C080919103C0919203D0919303109127
:104130009403811107C0C11175C0D11173C0111151
:1041400071C074C09F3F19F09F5F90938F03181642
:1041500024F40E94791E809391038091910387FF3C
:1041600005C00E94791E8195809391031C1624F44A
:104170000E94791E809392038091920387FF05C06D
:104180000E94791E8195809392036091910366232A
:1041900031F1C0919203CC2311F1062E000C770B64
:1041A000880B990B0E944C2523E333E343E35FE341
:1041B0000E94B0250E941425609391036C2FCC0FB0
:1041C000770B880B990B0E944C2523E333E343E3E1
:1041D0005FE30E94B0250E941425609392031D1690
:1041E00024F40E94C21E809393038091930387FF5F
:1041F00005C00E94C21E819580939303111624F47A
:104200000E94C21E809394038091940387FF05C08F
:104210000E94C21E819580939403DF91CF911F91DC
:104220000C94E81F9F3F09F08FCFA0CFDF91CF9173
:104230001F910895E0E9F3E085E0DF011D928A9582
:10424000E9F710928F0310928E0308958FE896E09D
:104250000E949A051F9281E08F931F9285E08F93B1
:1042600081E496E09F938F930E9433060F900F9006
:104270000F900F900F900F9008958330E9F128F47C
:10428000813061F0823009F10895853009F462C00F
:1042900008F449C0863009F474C00895809119016A
:1042A000262F30E0280F311D2F3F310524F4680FF1
:1042B0006093190103C08FEF809319018091190158
:1042C0001F928F938AE795E072C080911801262F84
:1042D00030E0280F311D2F3F310524F4680F609323
:1042E000180103C08FEF80931801809118011F926D
:1042F0008F9388E695E05BC080911701262F30E010
:10430000280F311D2F3F310524F4680F60931701EA
:1043100003C08FEF80931701809117011F928F9335
:1043200085E595E044C080911601262F30E0280FE6
:10433000311D2F3F310524F4680F6093160103C02F
:104340008FEF80931601809116011F928F9380E466
:1043500095E02DC080911501262F30E0280F311DEA
:104360002F3F310524F4680F6093150103C08FEFD0
:1043700080931501809115011F928F9387E295E03C
:1043800016C080911401262F30E0280F311D2F3FD9
:10439000310524F4680F6093140103C08FEF8093FC
:1043A0001401809114011F928F938CE095E09F93EC
:1043B0008F930E9433060F900F900F900F900895E7
:1043C000833081F128F4813059F08230D1F00895A2
:1043D000853009F449C0B8F1863009F456C0089513
:1043E00080911901681720F4861B8093190102C07F
:1043F00010921901809119011F928F938DEF94E013
:1044000054C080911801681720F4861B809318010E
:1044100002C010921801809118011F928F938BEEA9
:1044200094E043C080911701681720F4861B8093A5
:10443000170102C010921701809117011F928F93EC
:1044400088ED94E032C080911601681720F4861B35
:104450008093160102C010921601809116011F92DE
:104460008F9383EC94E021C080911501681720F4AC
:10447000861B8093150102C01092150180911501D1
:104480001F928F938AEA94E010C0809114016817FC
:1044900020F4861B8093140102C0109214018091B5
:1044A00014011F928F938FE894E09F938F930E9443
:1044B00033060F900F900F900F900895CF93C82F51
:1044C0001F928F9384E997E09F938F930E94330606
:1044D00081E090E0A0E0B0E0BC01CD0104C0660F37
:1044E000771F881F991FCA95D2F70E94321A0F9022
:1044F0000F900F900F90CF910C94AA12CF93873208
:10450000A8F58E3108F02BC1803109F49FC0F8F472
:10451000873009F464C0A8F4863009F024C1809182
:104520008603817F8E7F8093860389E997E00E94CE
:104530009A0583E89AE00E949A0581E080939603A9
:104540004CC08B30F1F18E3009F46CC00CC1863157
:1045500009F4B0C020F4813109F4EDC004C18931FF
:1045600009F491C08B3109F449C0FDC0883349F189
:1045700050F4893209F4F1C0853309F4EEC0873272
:1045800009F0F1C0EAC0833409F4E7C028F48A33A3
:1045900008F4E9C08953E4C0883409F0E4C00E94FB
:1045A000AA1282E79AE00E949A052FEF83ED90E32A
:1045B000215080409040E1F700C000000E941E1E84
:1045C0000CC080EC97E05CC089E59AE00E949A05F7
:1045D00080918603816080938603C1E0C9C0809189
:1045E0008603C82FC17080FFEFCF85E69AE00E9456
:1045F0009A0580918603817F8E7F3DC090918603CE
:1046000091FBCC27C0F981E0C827892FC0FB81F935
:1046100080938603CC2319F08CE49AE027C08EE3C4
:104620009AE02EC09091860392FBCC27C0F981E0DE
:10463000C827892FC0FB82F980938603CC2319F009
:104640008FE29AE013C08FE19AE01AC0909186033E
:1046500093FBCC27C0F981E0C827892FC0FB83F9E1
:1046600080938603CC2351F083E19AE00E949A055F
:10467000809186038160809386037AC086E09AE009
:104680000E949A05AACF87EF99E00E949A058EECC6
:1046900099E00E949A058CE899E00E949A0583E6C9
:1046A00099E00E949A0589E199E00E949A058EEEB0
:1046B00098E0E6CF80EE98E00E949A050E94FA0FFB
:1046C0001F928F9386EC98E09F938F930E943306FE
:1046D000809110011F928F938FEA98E09F938F93A0
:1046E0000E943306809189021F928F938CE998E093
:1046F0009F938F930E943306809111011F928F9395
:1047000089E898E09F938F930E9433060E94C31D0F
:104710009F938F937F936F9382E798E09F938F93FC
:104720000E9433068DB79EB746960FB6F8949EBF8B
:104730000FBE8DBF52CF0E94AA12C091110181E01D
:10474000C827C0931101CC2329F088E698E00E9485
:104750009A050EC08DE598E093CF80E001C08D51A1
:104760000E945E223ACF8BE598E00E949A05C0E055
:104770008C2FCF91089580E008950C94BB23CF93A4
:10478000C82F80919603813071F020F0823009F4B7
:104790004BC042C1E0911201F0911301808182323D
:1047A00009F03CC107C0E0911201F0911301808132
:1047B000823261F48C2F0E94BD23811104C08C2FA2
:1047C0000E947E222FC081E090E02CC08C2F0E949E
:1047D000BB23811126C0C431E1F070F4CB3081F0ED
:1047E000C031D1F40E9426218CE897E00E949A05FE
:1047F00082E08093960315C0C93259F0C83361F442
:1048000089E997E00E949A0580E997E00E949A055D
:1048100008C01092960304C18AE897E00E949A05A6
:10482000FFC081E08170FEC0C43228F5CE3108F0AF
:10483000C1C0CB30A1F1D0F4C73009F0D3C08EE1B4
:104840008093190182E3809318018AE08093170115
:1048500084E18093160188E08093150188E28093BB
:10486000140180E396E00E949A05BFC0C33149F16C
:10487000C431C1F0B7C0CB3409F4A9C028F4C9329F
:1048800089F0C83361F0AEC0C13509F49EC0C235AD
:1048900009F499C0CE3409F0A5C06AE09EC00E9418
:1048A0002621A3C080919503882319F010929503C7
:1048B0009CC08DE396E00E949A0581E08093960368
:1048C000B1C087E196E00E949A0585E096E00E94DB
:1048D0009A05809119011F928F9382E096E09F9331
:1048E0008F930E94330680E096E00E949A058EEE38
:1048F00095E00E949A05809118011F928F938BEE8C
:1049000095E09F938F930E94330689EE95E00E9475
:104910009A058AED95E00E949A05809117011F92F1
:104920008F9387ED95E09F938F930E94330685EDDB
:1049300095E00E949A0584EC95E00E949A0580918A
:1049400016011F928F9381EC95E09F938F930E94A5
:1049500033068FEB95E00E949A058AEA95E00E9463
:104960009A05809115011F928F9387EA95E09F9396
:104970008F930E94330685EA95E00E949A058EE89F
:1049800095E00E949A05809114011F928F938BE805
:1049900095E09F938F930E94330689E895E00E94EB
:1049A0009A058DB79EB748960FB6F8949EBF0FBE76
:1049B0008DBF1BC0CE51EC2FF0E0EC5CFE4F808130
:1049C0008093950312C061E003C061E006C06AE015
:1049D000809195030E943D2108C0809195030E941B
:1049E000E02103C08EE296E013C0809195038823F6
:1049F00069F01F928F9388E296E09F938F930E94B5
:104A000033060F900F900F900F9004C085E296E050
:104A10000E949A0581E006C01092960380E002C0D1
:104A200080E000CFCF9108950E941B256894B111BA
:104A30000C94AA2508950E948F2588F09F5798F01E
:104A4000B92F9927B751B0F0E1F0660F771F881F93
:104A5000991F1AF0BA95C9F714C0B13091F00E94AD
:104A6000A925B1E008950C94A925672F782F8827F0
:104A7000B85F39F0B93FCCF3869577956795B395D4
:104A8000D9F73EF490958095709561957F4F8F4F43
:104A90009F4F0895E89409C097FB3EF49095809548
:104AA000709561957F4F8F4F9F4F9923A9F0F92FF4
:104AB00096E9BB279395F695879577956795B79572
:104AC000F111F8CFFAF4BB0F11F460FF1BC06F5F58
:104AD0007F4F8F4F9F4F16C0882311F096E911C06A
:104AE000772321F09EE8872F762F05C0662371F08B
:104AF00096E8862F70E060E02AF09A95660F771F9F
:104B0000881FDAF7880F9695879597F9089557FDCE
:104B10009058440F551F59F05F3F71F04795880F2B
:104B200097FB991F61F09F3F79F0879508951216C2
:104B300013061406551FF2CF4695F1DF08C016166E
:104B400017061806991FF1CF86957105610508941F
:104B50000895E894BB2766277727CB0197F9089536
:104B60000E94C3250C9434260E94262638F00E9409
:104B70002D2620F0952311F00C941D260C9423264D
:104B800011240C94AA250E94872570F3959FC1F3E8
:104B9000950F50E0551F629FF001729FBB27F00DEB
:104BA000B11D639FAA27F00DB11DAA1F649F662740
:104BB000B00DA11D661F829F2227B00DA11D621F8F
:104BC000739FB00DA11D621F839FA00D611D221F49
:104BD000749F3327A00D611D231F849F600D211D2D
:104BE000822F762F6A2F11249F5750409AF0F1F0B0
:104BF00088234AF0EE0FFF1FBB1F661F771F881F19
:104C000091505040A9F79E3F510580F00C941D260D
:104C10000C94AA255F3FE4F3983ED4F386957795EC
:104C20006795B795F795E7959F5FC1F7FE2B880FBE
:104C3000911D9695879597F9089597F99F6780E854
:104C400070E060E008959FEF80EC089500240A94DE
:104C50001616170618060906089500240A94121657
:104C60001306140605060895092E0394000C11F48A
:104C7000882352F0BB0F40F4BF2B11F460FF04C037
:104C80006F5F7F4F8F4F9F4F089597FB072E16F44E
:104C9000009407D077FD09D00E945F2607FC05D05D
:104CA0003EF4909581959F4F0895709561957F4F43
:104CB0000895EE0FFF1F0590F491E02D0994AA1BB3
:104CC000BB1B51E107C0AA1FBB1FA617B70710F0F7
:104CD000A61BB70B881F991F5A95A9F78095909529
:0A4CE000BC01CD010895F894FFCF48
:104CEA000568010000FF5707E707C4078E075A0740
:104CFA00010164032808140A321E404D362239562F
:104D0A00030903D302B1027802EB0104021D023641
:0E4D1A00025602000102030405060708090004
:106800000000000000000000040005000600070072
:10681000080009000A000B000C000D000E000F001C
:1068200010001100120013001400150016001700CC
:10683000180019001A001B001C001D001E001F007C
:10684000200021002200230024002500260027002C
:10685000280000002A002B002C002D002E002F0005
:1068600030003100000033003400290036003700CA
:1068700038003900000000000000000000000000A7
:106880000000000000000000000000000000000008
:1068900000004900000000004C00000000004F0014
:1068A00050005100520000000000000000000000F5
:1068B00000000000000000000000000000000000D8
:1068C00000000000000000000000000000000000C8
:1068D00000000000000000000000000000000000B8
:1068E00000000000000000000000000000000000A8
:1068F000E000C2A2E200E300E400D2A2E600F1A3BD
:106900000000000000000000040005000600070071
:10691000080009000A000B000C000D000E000F001B
:1069200010001100120013001400150016001700CB
:10693000180019001A001B001C001D001E001F007B
:10694000200021002200230024002500260027002B
:10695000280000002A002B002C002D002E002F0004
:1069600030003100000033003400350036003700BD
:1069700038003900000000000000000000000000A6
:106980000000000000000000000000000000000007
:1069900000004900000000004C00000000004F0013
:1069A00050005100520000000000000000000000F4
:1069B00000000000000000000000000000000000D7
:1069C00000000000000000000000000000000000C7
:1069D00000000000000000000000000000000000B7
:1069E00000000000000000000000000000000000A7
:1069F000E000E100E200E300E400E500E600F1A4CD
:106A00000000000000000000010001000100010082
:106A1000010001000100010001000100010001006E
:106A2000010001000100010001000100010001005E
:106A3000010001000100010001000100010001004E
:106A4000010001000100010001000100010001003E
:106A5000010000000100010001000100010001002F
:106A600001000100000001000100350001000100EB
:106A70000100010000000000000000000000000014
:106A80000000000000000000000000000000000006
:106A900000000100000000000100000000000100F3
:106AA00001000100010000000000000000000000E3
:106AB00000000000000000000000000000000000D6
:106AC00000000000000000000000000000000000C6
:106AD00000000000000000000000000000000000B6
:106AE00000000000000000000000000000000000A6
:106AF000010001000100010001000100010001008E
:106B00000000000000000000EA4401000100E2442F
:106B10000100010001000100460001004A004B0095
:106B20000100010047004800028A0100E944010019
:106B30000100010001000100010001003A003B00DA
:106B40003C003D003E003F00400041004200430049
:106B5000010000000100390001004400450001006F
:106B60000100010000000100010035004D004E0051
:106B70000100010000000000000000000000000013
:106B80000000000000000000000000000000000005
:106B900000000100000000000100000000004D00A6
:106BA0004A004E004B000000000000000000000002
:106BB00000000000000000000000000000000000D5
:106BC00000000000000000000000000000000000C5
:106BD00000000000000000000000000000000000B5
:106BE00000000000000000000000000000000000A5
:106BF0000100010001000100650001000100F1A396
:106C00000000000000000000EA4401000100E2442E
:106C10000100010001000100460001004A004B0094
:106C20000100010047004800028A0100E944010018
:106C30000100010001000100010001003A003B00D9
:106C40003C003D003E003F00400041004200430048
:106C5000010000000100390001004400450001006E
:106C60000100010000000100010029004D004E005C
:106C70000100010000000000000000000000000012
:106C80000000000000000000000000000000000004
:106C900000000100000000000100000000004D00A5
:106CA0004A004E004B000000000000000000000001
:106CB00000000000000000000000000000000000D4
:106CC00000000000000000000000000000000000C4
:106CD00000000000000000000000000000000000B4
:106CE00000000000000000000000000000000000A4
:106CF0000100010001000100650001000100F1A494
:00000001FF
